:020000040800F2
:1000000000040020E1010008E3010008E30100080A
:10001000E3010008E3010008E3010008E301000830
:10002000E3010008E3010008E30100087D2E000859
:10003000E3010008E3010008E3010008E301000810
:10004000E3010008E3010008E3010008E301000800
:10005000E3010008E3010008DD3000080931000871
:1000600035310008613100088D310008E3010008D6
:10007000E3010008E3010008E3010008E3010008D0
:10008000E3010008E3010008E3010008E3010008C0
:10009000E3010008E3010008E3010008B9310008AA
:1000A000E3010008E3010008E3010008E3010008A0
:1000B000F92E0008E3010008E3010008E30100084D
:1000C000E3010008E3010008E3010008E301000880
:1000D000E3010008E3010008E3010008E301000870
:1000E00021320008E3010008E3010008E3010008F1
:1000F000E3010008E3010008E3010008E301000850
:10010000E3010008E3010008E3010008E30100083F
:10011000E3010008E3010008E3010008E30100082F
:10012000E3010008E3010008E3010008E30100081F
:10013000E3010008E3010008E3010008E30100080F
:10014000E3010008E3010008E3010008D1250008ED
:10015000E3010008E3010008E3010008E3010008EF
:10016000E3010008E3010008E3010008E3010008DF
:10017000E3010008E3010008E3010008E3010008CF
:10018000E3010008E3010008E3010008E3010008BF
:10019000E3010008E3010008E3010008E3010008AF
:1001A000E3010008E3010008E3010008E30100089F
:1001B000E3010008E3010008E3010008E30100088F
:1001C000E3010008E3010008E3010008E30100087F
:1001D000E3010008E3010008E3010008E30100086F
:1001E00002E000F000F8FEE772B6394880F30888B4
:1001F000384880F3098838484EF60851CEF200019D
:10020000086040F20000CCF200004EF63471CEF2ED
:1002100000010860BFF34F8FBFF36F8F40F2000003
:10022000C0F2F0004EF68851CEF200010860BFF334
:100230004F8FBFF36F8F4FF00000E1EE100A4EF6C4
:100240003C71CEF200010860062080F31488BFF3F1
:100250006F8F01F085FE02F0A7FD4FF055301F496A
:100260001B4A91423CBF41F8040BFAE71C49194A6A
:1002700091423CBF41F8040BFAE71A491A4A1B4B5A
:100280009A423EBF51F8040B42F8040BF8E70020F5
:100290001749184A91423CBF41F8040BFAE701F0B4
:1002A00063FE02F0DDFD144C144DAC4203DA54F849
:1002B000041B8847F9E700F03FF8114C114DAC42A0
:1002C00003DA54F8041B8847F9E701F04BBE00003D
:1002D000000400200024002000000008000000208E
:1002E00000040020503600080024002028240020AC
:1002F0002824002018340020E0010008E001000854
:10030000E0010008E00100082DE9F04F2DED108A12
:10031000C1F80CD0C3689D46BDEC108ABDE8F08FD3
:10032000002383F311882846A047002001F0A8FA93
:1003300001F058FA00DFFEE71A4B6FF07C0270B54F
:1003400000241A700F225C709C70DC701C715C7150
:100350009C71DC711C725C729A72DC7201F0D8FDC7
:10036000064601F0F7FD054650B90F4B9E4217D0E7
:1003700001339E4241F2883412BF05460024012514
:10038000002001F0CFFD0DB100F0B4F800F01EFD2B
:1003900000F002FC204600F00BF900F0ABF8F9E7A2
:1003A0000446EDE728240020010007B008B500F05E
:1003B00095FBA0F120035842584108BD07B5054BF5
:1003C00002211B88ADF8043001A800F0D5FB03B072
:1003D0005DF804FB1C330008064991F8243033B162
:1003E00000230822086A81F8243000F0F7BB0120BE
:1003F000704700BF482400202DE9F84F234C94F8A3
:1004000024300546884617468BBB2E46DFF87C9085
:10041000002F38D094F824A0BAF1000F05D1202283
:10042000FF214846266200F0BFFCCAF10805BD4224
:1004300028BF3D465FFA85FBAD0041462A4604EBE6
:100440008A0000F087FC94F82430A7EB0B079B444C
:100450005FFA8BFBBBF1080F2E44A844FFB284F86F
:1004600024B0D5D1FFF7B8FF0028D1D108E0266A23
:1004700006EB8306B042C9D0FFF7AEFF0028C4D117
:100480000020BDE8F88F0120BDE8F88F4824002047
:1004900010B5202383F311881248C3680BB101F013
:1004A00075FA0023104A0F484FF47A7101F032FABE
:1004B000002383F311880D4C236813B12368013B9B
:1004C0002360636813B16368013B6360084B1B786A
:1004D00033B9636823B9022000F032FC3223636031
:1004E00010BD00BF342400209104000878290020AA
:1004F0007024002010B5254B254953F8042F0132F4
:1005000000D110BD8B42F8D1224C234B22689A4275
:100510003AD9224B9B6803F1006303F580339A427A
:1005200032D2002000F052FB1D4B0220187000F068
:10053000FFFB1C4B1A6C00221A64196E1A66196EA6
:10054000596C5A64596E5A665A6E5A6942F0800262
:100550005A615A6922F080025A615A691A6942F056
:1005600000521A611A6922F000521A611B6972B6B0
:100570000D4A0E4B13601B682268202181F31188FD
:100580009D4683F30888104710BD00BFFCFF00089C
:100590001C00010804000108FFFF000828240020B7
:1005A000702400200038024008ED00E0000001083F
:1005B0002DE9F04FB04C97B020228146FF210EA8C4
:1005C000A66800F0F1FBAD4A1378A346A3B9AC4886
:1005D0000121C3601170202383F31188C3680BB11C
:1005E00001F0D4F90023A74AA5484FF47A7101F02D
:1005F00091F9002383F31188B9F1000F02D0A24BC7
:10060000C3F80090A14BA04A00241C7054602546FA
:1006100027469846012000F08BFBB9F1000F00F04F
:100620002282994B1B68002B40F01D8217B0BDE859
:10063000F08F0220FFF7BAFE002840F00E82944BA4
:100640001B88ADF82430022109A800F095FAE1E7F3
:100650004FF47A7000F042FA031E0193EFDB0220A0
:10066000FFF7A4FE82460028E9D0019B581E04280B
:1006700000F2F581DFE800F0030D1013160016A854
:10068000052340F8343D042100F076FA5446002753
:1006900052E004217848F7E704217E48F4E704217A
:1006A0007D48F1E71C24204600F092FA04340990BA
:1006B000042109A800F060FA2C2CF4D1E6E7002D03
:1006C000BDD0002CBBD00220FFF770FE05460028ED
:1006D00000F0C781012000F079FA022088F80000BC
:1006E00000F026FB0024E3B21846019300F07EFAE6
:1006F000824648B1019B184600F088FA0134002870
:10070000F1D12C46654B9BE70123022088F800308D
:1007100000F004FB5646DBF808309E4206D2304615
:1007200000F056FA0130ECD10436F4E7564B0026BF
:1007300088F800605E602C4600F03EFB1DB1002C86
:1007400018BF4FF00009FFF739FE63E7002D3FF4B3
:1007500076AF002C3FF473AF022088F8000000F061
:10076000E7FA322000F0BAF9B0F1000AC0F279815C
:100770001AF0030540F07581DBF8082006EB0A0348
:10078000934200F26E81BAF5807F00F26A81444B99
:10079000019355450DDA4FF47A7000F09FF90290FD
:1007A000029A002AC0F25D81019B029AEA54013547
:1007B000EEE7C820FFF7FAFD0546002800F051815A
:1007C0001F2E11D8C6F12004544528BF54460EAB45
:1007D00026F0030022463249184400F0BBFA2246B4
:1007E000FF212F4800F0E0FA4FEAAA0A5FFA8AF2E6
:1007F0002B493046FFF700FE0446002881D006EB67
:100800008A06054698E70220FFF7D0FD00283FF44E
:1008100016AFFFF7E1FD00283FF411AF002292462A
:10082000DBF808309A4259D21F2A1ED80E9B01339A
:100830001BD022F0030316A90B4453F8203C099364
:100840001848436883B3174800210DF1240E11F8AE
:100850000E3083EA0A03DBB2013150F82330042959
:1008600083EA1A2AF3D10432DAE71046019200F043
:10087000AFF9019A0990E3E72824002074250020AD
:1008800034240020910400087829002070240020DE
:100890001E3300082C2400203024002020330008C0
:1008A000742400207825002019464FF0080E11F01E
:1008B000010F4FEA51011FBF81F06D4181F43801F2
:1008C00081F4034181F02001BEF1010EEFD140F827
:1008D00023100133B3F5807FE6D1B4E716A80421D5
:1008E00040F84CAD00F048F926E716A8002340F880
:1008F000343D642100F01CF900287FF4A0AE0220F2
:10090000FFF754FD00283FF49AAE099800F090F9E3
:1009100016AB43F8480D04211846E3E716A8002358
:1009200040F8343D642100F003F900287FF487AEDD
:100930000220FFF73BFD00283FF481AE099800F04C
:1009400085F916AB43F8440DE5E70220FFF72EFDCD
:1009500000283FF474AE00F07FF916AB43F8400D69
:10096000D9E70220FFF722FD00283FF468AE09A96D
:10097000142000F077F9824616A8042140F83CAD17
:1009800000F0FAF8514609A8ACE7322000F0A6F8CA
:10099000B0F1000AFFF653AE1AF0030F7FF44FAE2A
:1009A000DBF808200AEB070393423FF648AE02202B
:1009B000FFF7FCFC00283FF442AE2AF0030ABA44D9
:1009C000BA453FF4B9AE384600F002F90421089068
:1009D00008A800F0D1F80437F2E74FF47A70FFF777
:1009E000E5FC00283FF42BAEFFF7F6FC00283FF4AF
:1009F00089AE0E9B01330CD008220EA90020FFF710
:100A0000FBFC00283FF47EAE2022FF210EA800F060
:100A1000CBF9FFF7D3FC304800F038FF06E616A804
:100A2000002340F8343D642100F082F8824600281B
:100A30007FF405AE0220FFF7B9FC00283FF4FFADBC
:100A4000FFF7BCFC41F2883000F020FF099800F06D
:100A5000E7F9D14600F0B0F9DCE505466CE6002781
:100A6000EDE52546EBE5002000F038F80290029B0A
:100A7000002BFFF6D2AD012000F050F9029B213B84
:100A8000122B3FF6C7AD01A252F823F0330600083F
:100A900051060008BF0600081506000815060008E4
:100AA000150600084D0700088B0900080708000814
:100AB000EB0800081D0900084B090008150600088E
:100AC0006309000815060008DB090008390700085B
:100AD000150600081F0A0008A086010037B5114B53
:100AE0001A780132D2B20024012A01468DF807405B
:100AF00011D80D4803681D6A4FF47A734B430122E5
:100B00000DF10701A847012805D1084B9DF8070002
:100B10001C7003B030BD4FF4FA7000F0B7FE4FF018
:100B2000FF30F6E700240020C82900208429002097
:100B300038B50E4B1A780132D2B2012A05460ED8CA
:100B40000B4803681C6A4FF47A734B43042229460E
:100B5000A047042803D1074B0020187038BD4FF47C
:100B6000FA7000F093FE4FF0FF3038BD00240020F3
:100B7000C82900208429002030B4054C2368DD6991
:100B8000044B0A46AC460146204630BC604700BFD5
:100B9000C8290020A086010070B501F0C1F8094CF9
:100BA000094E2070002530682378834208D901F06F
:100BB000B1F8336805440133B5F5803F3360F2D3B3
:100BC00070BD00BF852900208029002001F052B9A6
:100BD00000F1006000F580300068704700F10060AF
:100BE000920000F5803001F0DDB80000054B1A6876
:100BF000054B1B789B1A834202D9104401F08AB836
:100C000000207047802900208529002038B5074D35
:100C100004462868204401F085F828B92868204453
:100C2000BDE8384001F096B838BD00BF80290020EB
:100C300010F0030308D1B0F5007F05D800F1005093
:100C4000A0F508400068704700207047014BC0586D
:100C5000704700BF107AFF1F014B1868704700BF34
:100C6000002004E070B52A4B1C68C4F30B03240C6D
:100C700063B140F21342934231D040F219429342A1
:100C80002FD040F2214293422DD10323214A0C253B
:100C900005FB03235D6893F9082042F201039C429F
:100CA00024D0B4F5805F23D041F201039C4221D0CF
:100CB00041F203039C421FD041F207039C4208BF4C
:100CC0003122441E0C44013D0B46A3421ED215F9AD
:100CD000016F581C96B1034600F8016CF5E701233B
:100CE000D4E70223D2E73F220B4DD6E73322E3E7D6
:100CF0004122E1E75A22E4E75922E2E72C25844227
:100D00001D7001D9981C5A70401A70BD1846FBE737
:100D1000002004E03033000824330008022802BF1A
:100D2000024B4FF400129A61704700BF000402406A
:100D3000022802BF014B20229A6170470004024042
:100D4000022801BF024A536983F0200353617047B0
:100D50000004024010B50023934203D0CC5CC4547D
:100D60000133F9E710BD000030B5441E14F9010F3E
:100D70000B4660B193F90050854201F1010106D1A3
:100D80001AB993F90020801A30BD013AEEE7002A23
:100D9000F7D1104630BD000002460346981A13F9F9
:100DA000011B0029FAD1704702440346934202D046
:100DB00003F8011BFAE77047024B1A78024B1A70CE
:100DC000704700BF842900200024002038B5104D52
:100DD000104C284600F0A2F82146284600F0CAF838
:100DE00024680D48626DD2F8043843F00203C2F85B
:100DF000043800F04BFD0949204600F0C7F9626D48
:100E0000D2F8043823F00203C2F8043838BD00BF1A
:100E1000C8290020FC33000840420F002434000899
:100E200070470000026843681143016003B118472E
:100E30007047000013B5446BD4F894341A681178E5
:100E4000042915D1217C022912D119791289012393
:100E50008B4013420CD101A904F14C0001F01EFE9D
:100E6000D4F89444019B21790246206800F0DAF915
:100E700002B010BD143001F0A1BD00004FF0FF33EF
:100E8000143001F09BBD00004C3001F073BE000037
:100E90004FF0FF334C3001F06DBE0000143001F014
:100EA0006FBD00004FF0FF31143001F069BD00004C
:100EB0004C3001F03FBE00004FF0FF324C3001F0EB
:100EC00039BE0000D0F8942438B513681978042985
:100ED000054601D0012038BD017C0229FAD11279E2
:100EE0005C89012090400440F4D105F1140001F028
:100EF00001FD02460028EDD0D5F894544FF48073DC
:100F00002868697900F07CF9204638BD406BFFF70E
:100F1000D9BF000000207047704700007FB5124B1A
:100F20000360002343608360C360012502260F4BEA
:100F3000057404460290019300F18402294600964C
:100F40004FF48073143001F0B1FC094B019302940B
:100F500000964FF4807304F52372294604F14C0087
:100F600001F078FD04B070BD803300080D0F00085B
:100F7000350E00080B68202282F311880A7903EBF2
:100F8000820290614A79093243F822008A7912B1CB
:100F900003EB8203986102230374C0F894140023C6
:100FA00083F311887047000038B5037F044613B1FE
:100FB00090F85430ABB9201D01250221FFF732FF14
:100FC00004F1140025776FF0010100F087FC84F82C
:100FD000545004F14C006FF00101BDE8384000F0BE
:100FE0007DBC38BD10B5012104460430FFF71AFF5F
:100FF0000023237784F8543010BD000038B5044630
:101000000025143001F06AFC04F14C00257701F052
:1010100039FD201D84F854500121FFF703FF2046BD
:10102000BDE83840FFF74EBF90F8443003F060034E
:10103000202B19D190F84520212A0AD0222A4FF0DE
:1010400000030ED0202A0FD1084A82630722C26310
:1010500004E0064B83630723C3630023036401207A
:1010600070478363C363F9E70020704701240020C1
:10107000D0F8943437B51A681178042904461AD187
:10108000017C022917D11979128901238B4013425F
:1010900011D100F14C05284601F0B4FD58B101A969
:1010A000284601F0FBFCD4F89444019B21790246C8
:1010B000206800F0B7F803B030BD000000EB8103FA
:1010C000F7B59C6905460E46F4B1202383F31188D9
:1010D00005EB8607201D0821FFF7A4FEFB685B696E
:1010E0001B684C3413B1204601F0E6FC01A92046F0
:1010F00001F0D4FC024648B1019B3146284600F07D
:1011000091F8002383F3118803B0F0BDFB685A699E
:101110001268002AF5D01B8A013B1340F1D105F17A
:101120004402EAE7093138B550F82140DCB1202308
:1011300083F31188D4F894241368527903EB820363
:10114000DB689B695D6845B104216018FFF76AFEA2
:10115000294604F1140001F0D7FB2046FFF7B2FE48
:10116000002383F3118838BD7047000000F082BF70
:101170000123037000234360C36183620362C3627F
:1011800043620363038143817047000038B504461E
:10119000202383F3118800254160C5600561456106
:1011A000856100F077FF0223237085F3118838BD35
:1011B00070B500EB810305465069DA600E461446AF
:1011C00018B110220021FFF7EFFDA06918B110221D
:1011D0000021FFF7E9FD31462846BDE8704001F0E7
:1011E00023B80000028902F001020281428902F064
:1011F00001024281002202614261826101F0A8B8CD
:10120000F0B400EB81044789E4680125A4698D40AE
:101210003D43458123600023A2606360F0BC01F080
:10122000C3B80000F0B400EB81040789E46801252D
:1012300064698D403D43058123600023A2606360A3
:10124000F0BC01F03DB9000070B502230025044652
:101250000370A0F84C5080F84E5080F84F50058134
:101260004581C56005614561856180F8345000F0B5
:1012700077FF63681B6823B129462046BDE87040AC
:10128000184770BD436802781B6880F8502005221B
:1012900002700BB10421184770470000436890F8B2
:1012A00050201B6802700BB10521184770470000E1
:1012B00090F8343070B5044613B1002380F8343010
:1012C00004F14402204601F065F863689B6863BB43
:1012D00094F8445015F0600615D194F8453005F0A7
:1012E0007F0545EA032540F202339D4200F00E815E
:1012F0005BD8022D00F0DC803FD8002D00F0878005
:10130000012D00F0CF800021204601F09BFA002142
:10131000204601F08DFA63681B6813B10621204650
:101320009847062384F8343070BD2046984700283B
:10133000CED094F84B2094F84A3043EA0223E26B73
:10134000934238BFE36394F94430E56B002B4FF0D0
:10135000200380F2FD80002D00F0EC80092284F84B
:10136000342083F311880021E36BA26B2046FFF742
:1013700059FF002383F3118870BDB5F5817F00F01C
:10138000B180B5F5407F49D0B5F5807FBBD194F8E9
:101390004630012BB7D1B4F84C3023F00203A4F847
:1013A0004C30A663E6632664C3E740F201639D42C6
:1013B0001ED8B5F5C06F3BD2B5F5A06FA3D1B4F878
:1013C0004430B3F5A06F0ED194F8463084F84E3017
:1013D000204600F01DFF63681B6813B10121204601
:1013E0009847032323700023A363E3632364A0E7E8
:1013F000B5F5106F32D040F602439D4252D0B5F59C
:10140000006F80D104F14F03A363012324E004F1B2
:101410004C03A3630223E36325648AE794F8463010
:10142000012B7FF470AFB4F84C3043F00203B6E701
:1014300094F84920616894F848304D6894F8471052
:1014400043EA0223204694F84620A84700283FF4A8
:101450005AAF4368A3630368E363A4E72378042BCC
:1014600010D1202383F311882046FFF7BBFE86F3BB
:101470001188636884F84F601B68032121700BB1E9
:101480002046984794F84630002BACD084F84F3073
:101490000423237063681B68002BA4D0022120461C
:1014A0009847A0E7374BA3630223E36300239DE73C
:1014B00094F8481011F0800F204601F00F010ED073
:1014C00000F05AFF012806D002287FF41CAF2E4BF3
:1014D000A363E06367E72D4BA363E56363E700F075
:1014E0003DFFEFE794F84630002B7FF40CAF94F803
:1014F000483013F00F013FF476AF1A06204602D5AC
:1015000001F0B4F96FE701F0A7F96CE794F8463001
:10151000002B7FF4F8AE94F8483013F00F013FF43D
:1015200062AF1B06204602D501F08CF95BE701F0A3
:101530007FF958E7142284F8342083F311882B466E
:101540002A4629462046FFF75BFE85F3118870BDC9
:101550005DB1152284F8342083F311880021E36BF8
:10156000A26B2046FFF74CFE03E70B2284F83420E1
:1015700083F311882B462A4629462046FFF752FE60
:10158000E3E700BFB0330008A8330008AC3300081D
:1015900038B590F834300446152B29D8DFE803F02D
:1015A0003E28282828283E28280B2939282828289A
:1015B000282828283E3E90F84B1090F84A20C36B0C
:1015C00042EA01229A4214D9C268128AB3FBF2F5A8
:1015D00002FB15356DB9202383F311882B462A466B
:1015E0002946FFF71FFE85F311880A2384F834305B
:1015F00038BD142384F83430202383F3118800236A
:101600001A4619462046FFF7FBFD002383F3118895
:1016100038BD036C03B198470023E7E7002101F0D0
:1016200011F90021204601F003F963681B6813B12A
:101630000621204698470623D8E7000090F834207A
:10164000152A38B5044622D80123934040F641625A
:1016500013421DD113F480150FD19B0217D50B2314
:1016600080F83430202383F311882B462A462946FC
:10167000FFF7D8FD85F3118838BDC3689B695B68A7
:101680002BB9036C03B19847002384F8343038BD7C
:10169000002101F0D7F80021204601F0C9F8636865
:1016A0001B6813B10621204698470623EDE700008A
:1016B000024B00221B605B609A6070478829002003
:1016C000002303748268054B1B6899689142FBD222
:1016D0005A68036042601060586070478829002093
:1016E00008B5202383F31188037C032B05D0042B3A
:1016F0000DD02BB983F3118808BD436900221A600D
:101700004FF0FF334361FFF7DBFF0023F2E790E880
:101710000C001A6002685360F2E7000000230374B3
:101720008268054B1B6899689142FBD85A68036030
:10173000426010605860704788290020054B196985
:101740000874186802681A605360186101230374F2
:10175000FEF7DABD8829002030B54B1C87B005465E
:101760000A4C10D023690A4A01A800F0D3F8284691
:10177000FFF7E4FF049B13B101A800F007F9236908
:10178000586907B030BDFFF7D9FFF8E78829002076
:10179000E116000838B50C4D41612B6981689A68E3
:1017A0009142044603D8BDE83840FFF789BF184688
:1017B000FFF786FF01232C61014623742046BDE814
:1017C0003840FEF7A1BD00BF88290020044B1A68ED
:1017D0001B6990689B68984294BF00200120704765
:1017E0008829002010B5084C236820691A682260F7
:1017F0005460012223611A74FFF790FF01462069AB
:10180000BDE81040FEF780BD8829002082600222DA
:1018100002740022427470478368A3F17C0243F88B
:101820000C2C026943F83C2C426943F8382C074AD7
:1018300043F81C2CC26843F8102C022203F8082C31
:10184000002203F8072CA3F11800704721030008B9
:1018500010B5202383F31188FFF7DEFF0021044633
:10186000FFF798FF002383F31188204610BD000086
:10187000024B1B6958610F20FFF760BF88290020C9
:10188000202383F31188FFF7F3BF000008B501465A
:10189000202383F311880820FFF75EFF002383F3E2
:1018A000118808BD49B1064B42681B6918605A602F
:1018B000136043600420FFF74FBF4FF0FF307047C5
:1018C000882900200368984206D01A680260506098
:1018D00059611846FFF7F4BE7047000038B504465A
:1018E0000D462068844200D138BD036823605C60E7
:1018F0004561FFF7E5FEF4E7054B03F114025A6179
:101900009A614FF0FF32DA6100221A62704700BF1D
:1019100088290020F8B503614FF08043C2605C6AFB
:10192000194B1A46022952F8145F38BF022195421A
:1019300006461F460AD1586198611C6205604560E1
:1019400081600819BDE8F84001F07EB9186AAB68FB
:10195000241A0C1902D3E41A2D6804E09C4202D226
:10196000204401F07FF9AB689C42F4D86B68736047
:1019700035601E606E60B460A9684FF0FF33091BCC
:10198000A960FB61F8BD00BF8829002010B41B4C82
:10199000234653F8141F814210D0416802680A6040
:1019A000026851609A424FF00001C16003D0936811
:1019B00081680B4493605DF8044B70470A6862616C
:1019C00000209A425360C86003D15DF8044B01F0D7
:1019D00043B993688868034493604FF08042206A5B
:1019E000526A121A9342E6D9991A012998BF931C98
:1019F00018445DF8044B01F035B900BF8829002078
:101A000000207047FEE70000704700004FF0FF30F5
:101A100070470000022906D0032906D00129064894
:101A200018BF0020704705487047032A9ABF044832
:101A300000EBC200002070478034000834340008F6
:101A40000824002070B59AB001AD06460846294624
:101A5000144600F095F82846FFF79EF9C0B2431CE3
:101A60005B0086E8180023700323637000230234B0
:101A70001946DAB2904204F1020401D81AB070BDDE
:101A8000EA5C04F8022C04F8011C0133F1E70000C1
:101A900008B5202383F311880348FFF7E9FA0023F0
:101AA00083F3118808BD00BFC829002010B5044683
:101AB000052916D8DFE801F016150316161D202398
:101AC00083F311880E4A0121FFF772FB20460D4A6D
:101AD0000221FFF76DFB0C48FFF790FA002383F318
:101AE000118810BD202383F311880748FFF75CFAA3
:101AF000F4E7202383F311880348FFF773FAEDE737
:101B0000B4330008D8330008C829002038B50C4D7C
:101B10000C4C0D492A4604F10800FFF793FF05F12C
:101B2000CA0204F110000949FFF78CFF05F5CA72DB
:101B300004F118000649BDE83840FFF783BF00BF35
:101B4000902E002008240020043400080E340008E1
:101B50001934000870B5044608460D46FFF71CF915
:101B6000C6B22046013403780BB9184670BD324620
:101B70002946FFF7F9F80028F3D1012070BD0000D5
:101B80002DE9F84F05460C46FFF706F92B49C6B27A
:101B90002846FFF7DFFF08B10536F6B22849284688
:101BA000FFF7D8FF08B11036F6B2632E0DD8DFF874
:101BB0008C80DFF88C90234FDFF890A0DFF890B096
:101BC0002E7846B92670BDE8F88F29462046BDE834
:101BD000F84F01F09BBB252E2CD107224146284609
:101BE000FFF7C2F858B9DBF800302360DBF80430A7
:101BF0006360DBF80830A36007350C34E0E70822A7
:101C000049462846FFF7B0F8A0B90F4BA21C13F8BD
:101C1000011F09095345C95D02F8021C197801F03A
:101C20000F0102F10202C95D02F8031CEFD1183462
:101C30000835C5E7267001350134C1E7A034000836
:101C400019340008B53400080F7AFF1F1B7AFF1FF4
:101C5000A8340008BFF34F8F024AD368DB03FCD4DB
:101C6000704700BF003C024008B5094B1B7873B9B0
:101C7000FFF7F0FF074B1A69002ABFBF064A5A60F8
:101C800002F188325A601A6822F480621A6008BD34
:101C9000EE300020003C02402301674508B50B4BA5
:101CA0001B7893B9FFF7D6FF094B1A6942F000423F
:101CB0001A611A6842F480521A601A6822F480523B
:101CC0001A601A6842F480621A6008BDEE30002083
:101CD000003C02400B2870B513D80B4A0B4C13780C
:101CE00063B90B4E4FF0006144F8231056F82350AF
:101CF00001330C2B2944F7D10123137054F8200031
:101D000070BD002070BD00BF20310020F0300020E9
:101D1000C8340008014B53F820007047C83400084D
:101D20000C2070470B2810B5044601D9002010BDC7
:101D3000FFF7D0FF064B53F824301844C21A0BB9F2
:101D4000012010BD12680132F0D1043BF6E700BF5C
:101D5000C83400080B2810B504461ED8FFF77AFFD8
:101D6000FFF782FF0E49F323CB60FFF773FFC30039
:101D7000DBB243F4007343F002030B610B6943F4DD
:101D800080330B61FFF766FFFFF7A4FFFFF786FFC5
:101D90002046BDE81040FFF7C5BF002010BD00BFC2
:101DA000003C02402DE9F84312F00103154643D1EF
:101DB0000244B2F1016F3FD22C4B1B6813F00103B8
:101DC0003AD02B4CFFF750FFF323E360FFF742FFBD
:101DD00040F20127032D16D8254C0F46401A40F239
:101DE0000118EB1B0B44012B00EB0706236926D8D7
:101DF00023F001032361FFF751FF0120BDE8F883C1
:101E0000043D0430E6E78307E6D1236923F44073F9
:101E1000236123693B43236151F8046B0660BFF3E0
:101E20004F8FFFF717FF03689E42E9D0236923F025
:101E300001032361FFF732FF0020BDE8F88323F49C
:101E400040732361236943EA08032361B94637F8E5
:101E5000023B3380BFF34F8FFFF7FCFE3688B9F8A3
:101E60000030B6B2B342BCD0E0E700BF0038024059
:101E7000003C0240084908B50B7828B153B9FFF778
:101E8000F3FE01230B7008BD23B1BDE808400870C4
:101E9000FFF704BF08BD00BFEE30002010B50244BC
:101EA000064B0439D2B2904200D110BD441C00B29E
:101EB00053F8200041F8040FE0B2F4E75028004046
:101EC000104B30B51C6F240407D41C6F44F400740D
:101ED0001C671C6F44F400441C670B4C236843F4DC
:101EE000807323600244094B0439D2B2904200D17E
:101EF00030BD441C00B251F8045F43F82050E0B2FA
:101F0000F4E700BF00380240007000405028004055
:101F100007B5012201A90020FFF7C0FF019803B017
:101F20005DF804FB07B502A9012241F8040D002069
:101F3000FFF7C6FF03B05DF804FB0000034B1B680E
:101F40009B0042BF024B01221A7070477438024056
:101F500021310020014B1878704700BF213100204B
:101F600070470000FEE70000084A094B09498B4210
:101F700004D3094A0021934205D3704752F8040F55
:101F800043F8040BF3E743F8041BF4E77436000846
:101F9000183400201834002018340020836D30B528
:101FA00000229D68446D11464FF0FF3004EB421350
:101FB00001329542C3F80019C3F81019C3F8080993
:101FC000C3F8001BC3F8101BC3F8080BEED24FF088
:101FD0000113C4F81C3830BD890141F020010161B2
:101FE00003699B06FCD4122000F0C4BE204B03EB17
:101FF00080022DE9F047D2F80CE05D6DDEF8142088
:10200000461CD2F800C005EB063605EB40185168B7
:1020100061450BD3D5F83428012303FA00F022EAF6
:102020000000C5F834081846BDE8F087BEF8104037
:10203000ACEB0103A34228BF2346D8F81849A4B249
:10204000B3EB840F10D894681F46A4F1040959F823
:1020500004AFC6F800A0042F01D9043FF7E71C44E1
:102060000B4494605360D2E70020BDE8F08700BFC6
:102070002431002010B5054C2046FFF779F84FF0C9
:10208000A0436365024BA36510BD00BF243100204F
:102090001C3500080378012B70B5054650D12A4B3A
:1020A000446D98421BD1294B5A6B42F080025A630F
:1020B0005A6D42F080025A655A6D5A6942F08002A8
:1020C0005A615A6922F080025A610E2143205B69ED
:1020D00000F0D6FB1E4BE3601E4BC4F80038002313
:1020E000C4F8003EC02323606E6D4FF40413A36355
:1020F0003369002BFCDA012333610C2000F03AFE37
:102100003369DB07FCD4122000F034FE3369002B66
:10211000FCDA0026A6602846FFF740FF6B68C4F88B
:102120001068DB68C4F81468C4F81C684BB90A4B23
:10213000A3614FF0FF336361A36843F00103A36021
:1021400070BD064BF4E700BF243100200038024088
:102150004014004003002002003C30C0083C30C066
:10216000F8B5446D054600212046FFF735FFA96DFF
:1021700000234FF001128F68C4F834384FF0006626
:10218000C4F81C284FF0FF3004EB431201339F4288
:10219000C2F80069C2F8006BC2F80809C2F8080B5F
:1021A000F2D20B686A6DEB656362102313611669E6
:1021B00016F01006FBD1122000F0DCFDD4F8003838
:1021C00023F4FE63C4F80038A36943F4402343F0CA
:1021D0001003A3610923C4F81038C4F814380A4B5B
:1021E000EB604FF0C043C4F8103B084BC4F8003B11
:1021F000C4F81069C4F80039EB6D03F1100243F420
:102200008013EA65A362F8BDF8340008408000102E
:10221000426D90F84E10D2F8003823F4FE6343EA82
:102220000113C2F8003870472DE9F0410EB200EBFF
:1022300086080D46D8F80C100F6807F00303022B30
:1022400050D0032B50D03D4A3D4F012B18BF1746AD
:10225000446D4FEA451E04EB0E030022C3F8102B19
:102260008A6905F1100C002A40D04A8A05F158030A
:102270005B013A43E2500123D4F81C2803FA0CF323
:102280001343A6444A69C4F81C380023CEF8103919
:1022900005F13F03002A39D00A8A898B9208012967
:1022A00088BF4A43C16D04EB8303561841EA0242DA
:1022B000C66529465A602046FFF78EFED8F80C30D6
:1022C0001B8A43EA85531F4305F148035B01E7502E
:1022D0000123D4F81C2803FA05F51543C4F81C584B
:1022E000BDE8F081174FB3E7174FB1E704EB461392
:1022F000D3F8002B22F40042C3F8002BD4F81C289A
:10230000012303FA0CF322EA0303BAE704EB830385
:102310000E4A5A6004EB461629462046FFF75CFE3B
:10232000D6F8003923F40043C6F80039D4F81C3835
:10233000012202FA05F523EA0505CFE70080001027
:10234000008004100080081000800C1000040002BF
:10235000826D1268C265FFF721BE00005831436DDF
:1023600049015B5813F4004004D013F4001F14BF5C
:1023700001200220704700004831436D49015B583D
:1023800013F4004004D013F4001F14BF01200220F6
:102390007047000000EB8101CB68196A0B6813607D
:1023A0004B6853607047000000EB810330B5DD6877
:1023B000AA691368D36019B9402B84BF4023136006
:1023C0006B8A1468426D1C44013CB4FBF3F4634314
:1023D000033323F0030302EB411043EAC44343F009
:1023E000C043C0F8103B2B6803F00303012B09B274
:1023F0000ED1D2F8083802EB411013F4807FD0F8E8
:10240000003B14BF43F0805343F00053C0F8003B3F
:1024100002EB4112D2F8003B43F00443C2F8003B08
:1024200030BD00002DE9F041244D6E6D06EB4013E8
:102430000446D3F8087BC3F8087B38070AD5D6F8DA
:102440001438190706D505EB84032146DB682846B6
:102450005B689847FA072FD5D6F81438DB072BD5D9
:1024600005EB8403D968CCB98B69488A5E68B6FBF2
:10247000F0F200FB12628AB91868DA6890420DD255
:10248000121A83E81400202383F311880B48214695
:10249000FFF78AFF84F31188BDE8F081012303FA76
:1024A00004F26B8923EA02036B81CB6823B12146D6
:1024B0000248BDE8F0411847BDE8F0812431002012
:1024C00000EB810370B5DD68436D6C692668E660DA
:1024D0004A0156BB1A444FF40020C2F810092A687A
:1024E00002F00302012A0AB20ED1D3F8080803EB66
:1024F000421410F4807FD4F8000914BF40F08050DB
:1025000040F00050C4F8000903EB4212D2F8000971
:1025100040F00440C2F80009D3F83408012202FA5E
:1025200001F10143C3F8341870BD19B9402E84BFBE
:102530004020206020682E8A841940F00050013C21
:102540001A44B4FBF6F440EAC440C6E7F8B50446C2
:102550001E48456D05EB4413D3F80869C3F80869B4
:10256000F10717D5D5F81038DA0713D500EB840337
:10257000D9684B691F68DA68974218D2D21B0027C6
:102580001A605F60202383F311882146FFF798FFCC
:1025900087F31188330617D5D5F834280123A340D3
:1025A000134211D02046BDE8F840FFF71FBD0123BC
:1025B00003FA04F2038923EA020303818B68002BE8
:1025C000E8D021469847E5E7F8BD00BF2431002058
:1025D00096482DE9F84F456D6E69AB691E4016F4BB
:1025E000805F6E61044605D0FEF72EFEBDE8F84F11
:1025F00000F054BC002E12DAD5F8003E8B489B0741
:102600001EBFD5F8003E23F00303C5F8003ED5F801
:10261000043823F00103C5F80438FEF73FFE370500
:1026200002D58248FEF72EFEB0040CD5D5F8083846
:1026300013F0060FEB6823F470530CBF43F41053F0
:1026400043F4A053EB60310704D56368DB680BB13A
:1026500076489847F2025AD4B3020CD5D4F8548085
:10266000DFF8C8A100274FF00109A36D9B68F9B2FC
:102670008B4280F08780F70619D5616D0A6AC2F334
:102680000A1702F00F0302F4F012B2F5802F00F0E7
:10269000A180B2F5402F0AD104EB830301F58051EC
:1026A000DB68186A00231A469F4240F08780300397
:1026B000D5F8184813D5E10302D50020FFF7B2FE84
:1026C000A20302D50120FFF7ADFE630302D502206D
:1026D000FFF7A8FE270302D50320FFF7A3FE75032B
:1026E00084D5E00702D50020FFF730FFA10702D50F
:1026F0000120FFF72BFF620702D50220FFF726FF1C
:1027000023077FF573AF0320FFF720FF6EE7D4F8B0
:102710005480DFF818A100274FF00109A36D9B68D2
:102720005FFA87FB5B4597D308EB4B13D3F800297F
:1027300002F44022B2F5802F22D1D3F80029002ADA
:102740001EDAD3F8002942F09042C3F80029D3F8EA
:102750000029002AFBDB5946606DFFF73DFC22890A
:1027600009FA0BF322EA0303238104EB8B03DB68F2
:102770009B6813B15946504698475846FFF736FCB8
:102780000137CBE708EB4112D2F8003B03F44023BA
:10279000B3F5802F10D1D2F8003B002B0CDA628900
:1027A00009FA01F322EA0303638104EB8103DB6886
:1027B000DB680BB150469847013756E79C0708BFC6
:1027C0000A68072B98BF027003F101039CBF120A2D
:1027D000013069E7023304EB830201F5805152684E
:1027E00090690268D0F808C04068A2EB000E002291
:1027F000104697420AD104EB830463689B699A6888
:102800003A449A605A6817445F6050E712F0030F29
:1028100008BF0868964588BF8CF8000002F10102E5
:1028200084BF000A0CF1010CE3E700BF2431002053
:10283000436D03EB4111D1F8003B43F40013C1F8A1
:10284000003B7047436D03EB4111D1F8003943F46D
:102850000013C1F800397047436D03EB4111D1F803
:10286000003B23F40013C1F8003B7047436D03EBBA
:102870004111D1F8003923F40013C1F80039704731
:1028800000F1604300F01F02400903F561430901B4
:102890008000C9B200F1604083F8001300F5614088
:1028A00001239340C0F880310360704730B5039C2A
:1028B0000172043304FB0325C361049B03630021FD
:1028C000059B00604060C1604261026185610462F5
:1028D00042628162C162436330BD00000022416AEE
:1028E00041610161C2608262C2626FF00101FEF764
:1028F000F5BF000003694269934203D1C2680AB17F
:1029000000207047181D704703691960C2680132C2
:10291000C260C269134482690361934224BF436A5F
:1029200003610021FEF7CEBF38B504460D46E368CB
:102930003BB16269131D1268A3621344E362002075
:1029400038BD237A33B929462046FEF7ABFF00286D
:10295000EDDA38BD6FF00100FBE70000C368C26923
:10296000013BC3604369134482694361934224BFBE
:10297000436A436100238362036B03B118477047C6
:1029800070B52023044683F31188866A3EB9FFF7A9
:10299000CBFF054618B186F31188284670BDA36A9F
:1029A000E26A13F8015BA362934202D32046FFF769
:1029B000D5FF002383F31188EFE700002DE9F84FDE
:1029C00004460E4690469946202787F31188002535
:1029D000AA46D4F828B0BBF1000F09D149462046D9
:1029E000FFF7A2FF20B18BF311882846BDE8F88FCE
:1029F000A16AE36AA8EB050B5B1A9B4528BF9B46BF
:102A0000BBF1400F1BD9334601F1400251F8040BD2
:102A100043F8040B9142F9D1A36A40334036A362D4
:102A20004035A26AE36A9A4202D32046FFF796FF36
:102A30008AF311884545D8D287F31188C9E7304613
:102A40005A46FEF787F9A36A5B445E44A3625D447D
:102A5000E7E7000010B5029C0172043303FB042178
:102A6000C36100238362C362039B0363049B006012
:102A70004060C460426102618161046242624363FA
:102A800010BD0000026AC260426A42610261002217
:102A90008262C2626FF00101FEF720BF43690269E2
:102AA0009A4203D1C2680AB100207047184650F814
:102AB000043B0B6070470000C368C2690133C36008
:102AC0004369134482694361934224BF436A43616B
:102AD0000021FEF7F7BE000038B504460D46E36856
:102AE0003BB123691A1DA262E2691344E36200202C
:102AF00038BD237A33B929462046FEF7D3FE002895
:102B0000EDDA38BD6FF00100FBE7000003691960E2
:102B1000C268013AC260C269134482690361934288
:102B200024BF436A036100238362036B03B1184728
:102B30007047000070B5202304460E4683F31188C9
:102B4000856A35B91146FFF7C7FF10B185F31188C3
:102B500070BDA36A1E70A36AE26A01339342A36246
:102B600004D3E16920460439FFF7D0FF002080F349
:102B7000118870BD2DE9F84F04460D4691469A46DE
:102B80004FF0200888F311880026B346A76A4FB992
:102B900051462046FFF7A0FF20B187F31188304649
:102BA000BDE8F88FA06AE76AA9EB06033F1A9F42C7
:102BB00028BF1F46402F1BD905F1400355F8042BB1
:102BC00040F8042B9D42F9D1A36A4033A3624036FA
:102BD000A26AE36A9A4204D3E16920460439FFF706
:102BE00095FF8BF311884E45D9D288F31188CDE734
:102BF00029463A46FEF7AEF8A36A3B443D44A36239
:102C00003E44E5E7026943699A4203D1C3681BB9B0
:102C1000184670470023FBE7836A002BF8D0043B7B
:102C20009B1AF5D01360C368013BC360C3691A44A3
:102C3000836902619A4224BF436A0361002383626D
:102C40000123E5E700F06CB94FF0804300225863A0
:102C50001A610222DA6070474FF080430022DA6086
:102C6000704700004FF0804358637047FEE7000054
:102C700010B5174CFEF71CFDFEF73EFE80221549ED
:102C80002046FEF7C3FD012344F8180C0374124BD1
:102C9000124AD96821F4E0610904090C0A43104979
:102CA000DA60CA6842F08072CA600E490A6842F06F
:102CB00001020A601022DA77202283F82220002302
:102CC00083F3118862B60848BDE81040FEF7C0BD26
:102CD000B02900202835000800ED00E00003FA05C7
:102CE000F0ED00E0001000E0303500082DE9F84F6D
:102CF0001F4C4FF00008656904F11407C1464FF0FE
:102D00008043266A5B6AAA689E1B96421DD34FF0D9
:102D1000200AAA68236AD5F80CB0134423622B68F2
:102D2000BB425F60A6EB02066361C5F80C8001D16F
:102D3000FFF792FF89F311882869D8478AF3118831
:102D40006569AB689E42E4D2D9E76269BA420CD0A9
:102D5000916823628E1B9660A86802282CBF181801
:102D6000981CBDE8F84FFFF77DBFBDE8F88F00BFA6
:102D700088290020034B59685A68521A9042FBD8A0
:102D8000704700BF001000E04B6843608B688360B1
:102D9000CB68C3600B6943614B6903628B69436213
:102DA0000B6803607047000008B5224B22481A697F
:102DB00040F2FF110A431A611A6922F4FF7222F0ED
:102DC00001021A611A691A6B0A431A631A6D0A43DF
:102DD0001A651A4A1B6D1146FFF7D6FF184802F113
:102DE0001C01FFF7D1FF174802F13801FFF7CCFFB4
:102DF000154802F15401FFF7C7FF144802F17001B2
:102E0000FFF7C2FF124802F18C01FFF7BDFF114826
:102E100002F1A801FFF7B8FF0F4802F1C401FFF764
:102E2000B3FF0E4802F1E001FFF7AEFFBDE8084036
:102E300000F0E0B8003802400000024050350008C1
:102E40000004024000080240000C02400010024052
:102E50000014024000180240001C02400020024002
:102E600008B500F037FAFFF703FFFFF767F8BDE892
:102E70000840FEF74BBE000070470000064A53684A
:102E800023F001035360EFF30983683383F3098868
:102E9000002383F31188704730EF00E010B5202342
:102EA00083F31188104B5B6813F4006318D0F1EEC4
:102EB000103AEFF309844FF0807344F84C3C0B4B0D
:102EC000DB6844F8083CA4F1680383F30988FEF743
:102ED0007DFC18B1064B44F8503C10BD054BFAE799
:102EE00083F3118810BD00BF00ED00E030EF00E07B
:102EF00031030008340300084FF0804310B51A690D
:102F0000920708D500241C61202383F31188FFF762
:102F1000EDFE84F31188BDE81040FFF7BFBF00004D
:102F2000104B1A6C42F001021A641A6E42F0010250
:102F30001A660D4A1B6E936843F0010393604FF0CD
:102F4000804353229A624FF0FF32DA6200229A6184
:102F50005A63DA605A6001225A6108211A601C2003
:102F6000FFF78EBC00380240002004E01F4B1A69B6
:102F70006FEAC2526FEAD2521A611A69C2F30802AA
:102F80001A614FF0FF301A695A69586100215A6975
:102F900059615A691A6A62F080521A621A6A02F01A
:102FA00080521A621A6A5A6A58625A6A59625A6A8E
:102FB0001A6C42F080521A641A6E42F080521A66FD
:102FC0001A6E0B4A106840F480701060186F00F49D
:102FD0004070B0F5007F1EBF4FF48030186719674E
:102FE000536823F40073536000F054B90038024072
:102FF00000700040304B4FF080521A642F4A4FF45B
:10300000404111601A6842F001021A601A68920782
:10301000FCD59A6822F003029A60274B19469A68F9
:1030200012F00C02FBD1186800F0F90018609A60E9
:103030001A6842F480321A600B689B03FCD54B6F10
:1030400043F001034B671C4B5A6F9007FCD51C4A99
:103050005A601A6842F080721A60184A536859041C
:10306000FCD5154B1A689201FCD5164A9A60164B8E
:103070001A68164B9A42164B1BD1164A1168164A0B
:10308000914216D140F205121A600B4B9A6842F039
:1030900002029A609A6802F00C02082AFAD15A6C6D
:1030A00042F480425A645A6E42F480425A665B6E21
:1030B000704740F20572E7E70038024000700040B8
:1030C0000854400700948838002004E01164002070
:1030D000003C024000ED00E041C20F41084A08B543
:1030E000536911680B4003F00103536123B1054A92
:1030F00013680BB150689847BDE80840FFF7CEBE93
:10310000003C014098330020084A08B55369116813
:103110000B4003F00203536123B1054A93680BB1DE
:10312000D0689847BDE80840FFF7B8BE003C0140B2
:1031300098330020084A08B5536911680B4003F022
:103140000403536123B1054A13690BB150699847D1
:10315000BDE80840FFF7A2BE003C014098330020C4
:10316000084A08B5536911680B4003F0080353611E
:1031700023B1054A93690BB1D0699847BDE808406F
:10318000FFF78CBE003C014098330020084A08B588
:10319000536911680B4003F01003536123B1054AD2
:1031A000136A0BB1506A9847BDE80840FFF776BE36
:1031B000003C014098330020174B10B55C691A6839
:1031C000144004F478725A61A30604D5134A936A32
:1031D0000BB1D06A9847600604D5104A136B0BB147
:1031E000506B9847210604D50C4A936B0BB1D06BFA
:1031F0009847E20504D5094A136C0BB1506C984707
:10320000A30504D5054A936C0BB1D06C9847BDE873
:103210001040FFF743BE00BF003C01409833002040
:103220001A4B10B55C691A68144004F47C425A6168
:10323000620504D5164A136D0BB1506D98472305EE
:1032400004D5134A936D0BB1D06D9847E00404D5B3
:103250000F4A136E0BB1506E9847A10404D50C4A67
:10326000936E0BB1D06E9847620404D5084A136F71
:103270000BB1506F9847230404D5054A936F0BB1E7
:10328000D06F9847BDE81040FFF708BE003C0140F2
:1032900098330020062108B50846FFF7F1FA062109
:1032A0000720FFF7EDFA06210820FFF7E9FA0621CB
:1032B0000920FFF7E5FA06210A20FFF7E1FA0621C7
:1032C0001720FFF7DDFA06212820BDE80840FFF7A8
:1032D000D7BA000008B5FFF749FE00F00BF8FDF77C
:1032E00045FFFDF719FEFFF7C7FDBDE80840FFF7F2
:1032F000A9BC0000002304491A465A50C8180833D4
:10330000802B4260F9D1704798330020034611F8B2
:10331000012B03F8012B002AF9D170471210121368
:103320001211000053544D3332463F3F3F0000001E
:1033300000000000243300083F00000013040000D8
:10334000603300083F000000190400006A330008E1
:103350003F00000021040000743300083F0000001B
:1033600053544D3332463430780053544D33324643
:103370003432780053544D33324634343658580082
:1033800000000000910E00087D0E0008B90E000834
:10339000A50E0008B10E00089D0E0008890E000859
:1033A000750E0008150F0008000000000100000065
:1033B000000000000200000000000000BD10000836
:1033C0002511000840004000602E0020702E0020D3
:1033D00002000000000000000300000000000000E8
:1033E000691100080000000010000000802E00207D
:1033F0000000000001000000000000002431002057
:10340000010102004172647550696C6F74002542BD
:103410004F415244252D424C002553455249414CC1
:1034200025000000AD1A0008151A00082910000830
:10343000911A0008430000003C34000809024300D0
:10344000020100C03209040000010202010005244B
:1034500000100105240100010424020205240600D5
:1034600001070582030800FF09040100020A0000A9
:10347000000705010240000007058102400000002E
:103480001200000088340008120110010200004000
:1034900083044057000201020301000004030904F1
:1034A00025424F41524425006F6D6E696275736607
:1034B0003470726F00303132333435363738394139
:1034C0004243444546000000004000000040000028
:1034D0000040000000400000000001000000020069
:1034E00000000200000002000000020000000200D4
:1034F000000002000000020000000000B1120008FD
:10350000911500083D16000840004000843100205D
:103510008431002001000000943100208000000070
:1035200040010000030000006D61696E00000000B2
:1035300048350008A0310020983300200100000029
:103540006D2C00080000000069646C65000000003C
:103550000000800200000000AAAAAAAA0000000041
:10356000FFFF00000000000000A00A0000040000AF
:1035700000000000AAAAAAAA00000000DFFF0000C5
:10358000000000000000000000000000000000003B
:10359000AAAAAAAA00000000FFFF00000000000085
:1035A000000000000000000000000000AAAAAAAA73
:1035B00000000000FFFF000000000000000000000D
:1035C0000000000000000000AAAAAAAA0000000053
:1035D000FFFF0000000000000000000000000000ED
:1035E00000000000AAAAAAAA00000000FFFF000035
:1035F00000000000000000000000000000000000CB
:10360000AAAAAAAA00000000FFFF00000000000014
:103610000000000000000000000000000A000000A0
:103620000000000003000000000000000000000097
:10363000000000000000000000000000000000008A
:10364000000000000000000000000000000000007A
:10365000FF00960000000008040000009C340008F1
:10366000000000000000000000000000000000005A
:08367000000000000000000052
:00000001FF
